:100000009728A4003B200C080D04031992288C208B
:1000100084132408800664000D280E288C0A031916
:100020008D0F0B28800692288F0026088400240953
:100030003C2084138F0803199228F03091000E0899
:1000400080389000F03091030319910003198F0359
:10005000031992282B283F2003010C1824088E1F17
:1000600024088E0803190301900F382880061F28E2
:10007000392800002228FF3A8417800592280D08AD
:100080000C0403198C0A80300C1A8D060C198D068D
:100090008C188D060D0D8C0D8D0D92288F018E0004
:1000A000FF308E07031C8F07031C922803308D003E
:1000B000DF305C2050288D01E83E8C008D09FC303B
:1000C000031C65288C07031862288C0764008D0FB9
:1000D00062280C186B288C1C6F2800006F28080001
:1000E0008D018F018E000230752894000F080D02DB
:1000F000031D7C280E080C0204300318013003197C
:1001000002301405031DFF3092280038031DFF3014
:100110000405031DFF3092288C098D098C0A0319F0
:100120008D0A0800831303138312640008008316EA
:10013000FF3085000C3086008312061383160613E9
:10014000831286128316861283120130AA0064007D
:1001500006302A020318CC280630A6001030A4006E
:1001600050308E000430142064308E000230142091
:1001700086108316861083120610831606103230FE
:1001800083124E208614831686108312061483165B
:1001900006108312AA0FA7280630A6001030A4006C
:1001A00064308E000430142078308E000230142029
:1001B00050308E00023014205A308E00023014204D
:1001C000861083168610831206108316061083127B
:1001D0006400051EF32806148316061083129E3051
:1001E000A9006621FA280610831606108312C8306B
:1001F000A90066216400851D0529861483168610D2
:1002000083129830A80053210C298610831686107B
:1002100083126430A80053210030851901308C000E
:10022000013070209E000030051A01308C00013032
:100230007020A0001E08840020088520A000A100D6
:10024000640020082104031938290130AA00640041
:1002500007302A02031833299630A8009F30A900DE
:100260003921AA0F27296430A800C830A9003921F4
:10027000E8280130AB00640010302B02031852292B
:1002800028088C008D0106308400403001202908A8
:100290008C008D01063084002030012006304E2075
:1002A000AB0F3B2908000130AC0064000B302C027E
:1002B0000318652928088C008D0106308400403021
:1002C000012006304E20AC0F552908000130AD004A
:1002D00064000B302D020318782929088C008D0149
:1002E000063084002030012006304E20AD0F6829F2
:0602F000080063007929FB
:02400E00F53F7C
:00000001FF
